:100000002FC0FECFFDCFFCCFFBCFFACFF9CFF8CF7B
:10001000F7CFF6CFF5CFF4CFF3CFF2CFF1CFF0CFCC
:10002000EFCFEECFEDCF1F111F121F101D151715AB
:10003000151F07041F17151D1F151D1905031F1573
:100040001F17151F0404040000000000000000003A
:1000500000002100600126000A00040048000000A2
:10006000F894EE27ECBBF1E0FBBFEBBFE5BFF8E196
:10007000F1BDE1BD8DE0A2E0BB27ED938A95E9F7E4
:1000800080E094E0A0E6ED930197E9F7E2E5F0E087
:1000900085919591009761F0A591B5910590159086
:1000A000BF01F00105900D920197E1F7FB01F0CF40
:1000B000EFE5EDBFE4E0EEBFC0E6D1E000C0E0E078
:1000C000E8BBE0ECE7BBE0E0E5BBE4BBE2BBEFE1B3
:1000D000E1BBE0E0E3BFE2BFEFBDEEBDEDBDECBDD7
:1000E000E7BDE6BDEBBDEABDE9BDE8BDE2BDE5BDEE
:1000F000E4BDE3BDE5BFE9BFE0E8E8B9E0E0E0BFAB
:10010000E0ECE7B9E6EEE6B9349BFECFC4B0D5B07B
:10011000E8EEF3E0CE16DF0690F0E4B3E03011F441
:10012000E0E11BC0E4B3E03111F4E0E216C0E4B357
:10013000E03229F4EAE07E2E6E2E9E2E23C0E4E605
:10014000F0E0CE16DF0650F4E4B3E03211F4E0E163
:1001500004C0E4B3E03111F4E0E0E4BBD601E4E62E
:10016000F0E0C1D09E2ED601E4E6F0E0CFD06F01E2
:10017000D601EAE0F0E0B7D06E2ED601EAE0F0E07A
:10018000C5D07E2EEFE1E1BBE0ECE7BBA92DB0E0EE
:10019000E3E0F0E0EA02F0014E2EE0E28E2EE0E035
:1001A000E8BB5524E3E05E1628F5E1B3EF71E829DA
:1001B000E1BBE4B3E03029F48F9B02C0C69A01C0D2
:1001C000C698A52DBB27E42DF0E0EA0FFB1FE05AEF
:1001D000FE4FE081E2BBE2E0F0E0FA93EA9377D0F1
:1001E000E0E0E2BBA82DB0E0FD01EE0FFF1F8E2E78
:1001F0005394D8CFEFE1E1BBA62DB0E0E3E0F0E00F
:10020000EA02F0014E2EE1E08E2EE0E0E8BB55243C
:10021000E3E05E1628F5E7B3E07CE829E7BBE4B34A
:10022000E03129F4BA9B02C0C79A01C0C798A52D36
:10023000BB27E42DF0E0EA0FFB1FE05AFE4FE08100
:10024000E2BBE2E0F0E0FA93EA9341D0E0E0E2BB07
:10025000A82DB0E0FD01EE0FFF1F8E2E5394D8CFD6
:10026000A72DB0E0E3E0F0E0EA02F0014E2E5524C5
:10027000E3E05E16E8F4E7B3E07CE829E7BBA52DF0
:10028000BB27E42DF0E0EA0FFB1FE05AFE4FE081B0
:10029000E2BBE2E0F0E0FA93EA9319D0E0E0E2BBDF
:1002A000A82DB0E0FD01EE0FFF1F8E2E5394E0CF7E
:1002B000E0ECE7BBAB2DB0E0E8E0F0E02AD0EA1BD1
:1002C000BE2EBB2009F05ECF369A1ECFFFCFE9913C
:1002D000F991309639F080ED97E00197F1F7A89504
:1002E0003197C9F708950024112490E1AA0FBB1F8C
:1002F000001C111C0E1A1F0A18F40E0E1F1E01C03E
:10030000A1609A9599F7FD01D0010895ECDFFD01F8
:1003100008951B2EBF2FF12D1A2EAE2FE12D08951B
:00000001FF
